:100000002500080C2400170C0A0963002E0B84013C
:100010006000A40284011F0E4307070A000836008F
:10002000D6004307180A1402240000022B001B0A02
:10003000030C35001D0A800C1E0A830C2C00A00C3A
:10004000C6042A00080C2800E6046A03C604030656
:10005000C6050000E605E802240A0000E6040000E8
:10006000C6050000000000000000E605C606EC041E
:10007000E604EC07610A0C020F0EE201450A480A89
:10008000610A450A4B0A500A610AAC020902210AB8
:10009000AC020B02210AE605C605AC02A10C200A3F
:1000A000C6050000E605080C2800E6050305C6079E
:1000B00003046B03E604C605E802550AE6050000E2
:1000C000E604C604E6050000000000000000C605C6
:1000D000140224000B0220000C0227000008FF0F6E
:1000E000FF0FFF0FFF0FFF0FFF0FFF0FFF0FFF0FA0
:1000F000FF0FFF0FFF0FFF0FFF0FFF0FFF0FFF0F90
:10010000FF0FFF0FFF0FFF0FFF0FFF0FFF0FFF0F7F
:10011000FF0FFF0FFF0FFF0FFF0FFF0FFF0FFF0F6F
:1001200063006F007000790072006900670068006A
:10013000740020006100650072006F0070006900AB
:10014000630020003200300030003000200020002A
:100150002000200020002000FF0FFF0FFF0FFF0FE7
:10016000FF0FFF0FFF0FFF0FFF0FFF0FFF0FFF0F1F
:10017000FF0FFF0FFF0FFF0FFF0FFF0FFF0FFF0F0F
:10018000FF0FFF0FFF0FFF0FFF0FFF0FFF0FFF0FFF
:10019000FF0FFF0FFF0FFF0FFF0FFF0FFF0FFF0FEF
:1001A000FF0FFF0FFF0FFF0FFF0FFF0FFF0FFF0FDF
:1001B000FF0FFF0FFF0FFF0FFF0FFF0FFF0FFF0FCF
:1001C000FF0FFF0FFF0FFF0FFF0FFF0FFF0FFF0FBF
:1001D000FF0FFF0FFF0FFF0FFF0FFF0FFF0FFF0FAF
:1001E000FF0FFF0FFF0FFF0FFF0FFF0FFF0FFF0F9F
:1001F000FF0FFF0FFF0FFF0FFF0FFF0FFF0FFF0F8F
:10020000FF0FFF0FFF0FFF0FFF0FFF0FFF0FFF0F7E
:10021000FF0FFF0FFF0FFF0FFF0FFF0FFF0FFF0F6E
:10022000FF0FFF0FFF0FFF0FFF0FFF0FFF0FFF0F5E
:10023000FF0FFF0FFF0FFF0FFF0FFF0FFF0FFF0F4E
:10024000FF0FFF0FFF0FFF0FFF0FFF0FFF0FFF0F3E
:10025000FF0FFF0FFF0FFF0FFF0FFF0F910C0200AB
:100260000B0C0600660070006E00020C2900110CD9
:100270003400000C0F0907023300020C2900110C96
:100280003400000C0F0907023300030C9100030631
:100290004B0B620C310069000F0C3400000C0F098D
:1002A000070233000F0291000306580B020C2F00C7
:1002B0006900A9020D0C3400000C0F09070233007D
:1002C0000D02C50F4306730B0D02E40F4306730BBB
:1002D000C50C2D006900A9023200120C3400010C7B
:1002E0000F09070233000607960B6606880B0D02FE
:1002F000C50F43077D0BE40C7E0BC50C2D00690078
:10030000A9023200120C3400010C0F09070233005D
:100310002606960B620C3100020C290011023200F5
:10032000120C3400010C0F09070233000D022100EA
:100330000606B10B2607AA0BB0021102D101330049
:10034000100293000306A80B860413023000AC0BC6
:100350008605AC0B700086042607A6042606A605B3
:10036000F60B000C4606010CEE010F028E00030690
:10037000BC0B8605A605BE0B8604A6040E02640F00
:100380004307F60B6E002606DD0B10024307D10B68
:100390006607F10BAF020F0291000306E80B110292
:1003A000E70B1002030F4307DD0B6606DD0B0F02A0
:1003B0003100020C29001102EA0B6606F10B100253
:1003C0004307F10BEF00CF004307E80B020C2F00AF
:1003D00069000F023200120C3400010C0F090702F1
:1003E0003300B0021002060F4306700001024307FB
:1003F000F60B040CA6010000960B0008FF0FFF0F80
:080400000F000F000F000F00B8
:021FFE00EA3FB8
:00000001FF
